:103800000C94341C0C944F1C0C944F1C0C944F1CA7
:103810000C944F1C0C944F1C0C944F1C0C944F1C7C
:103820000C944F1C0C944F1C0C944F1C0C944F1C6C
:103830000C944F1C0C944F1C0C944F1C0C944F1C5C
:103840000C944F1C0C944F1C0C944F1C0C944F1C4C
:103850000C944F1C0C944F1C0C944F1C0C944F1C3C
:103860000C944F1C0C944F1C11241FBECFEFD4E0BE
:10387000DEBFCDBF11E0A0E0B1E0ECE3FFE302C0AA
:1038800005900D92A230B107D9F712E0A2E0B1E0A5
:1038900001C01D92AD30B107E1F70C94311D0C94BD
:1038A000001CCF93DF93CDB7DEB724970FB6F89403
:1038B000DEBF0FBECDBF382F882309F433E010924E
:1038C0000A02332309F44BC020E02D9A19821A8290
:1038D0001B821C8289819A81AB81BC8180549F416B
:1038E000A040B040A0F489819A81AB81BC8101964F
:1038F000A11DB11D89839A83AB83BC8389819A8181
:10390000AB81BC8180549F41A040B04060F32D98B2
:1039100019821A821B821C8289819A81AB81BC81A7
:1039200080549F41A040B040A0F489819A81AB812E
:10393000BC810196A11DB11D89839A83AB83BC8391
:1039400089819A81AB81BC8180549F41A040B04065
:1039500060F32F5F231708F4B8CF20930A02249650
:103960000FB6F894DEBF0FBECDBFDF91CF910895A3
:10397000EF92FF920F931F93EE24FF248701809113
:10398000C00087FD17C00894E11CF11C011D111D2A
:1039900081E2E81681EAF80687E0080780E0180768
:1039A00070F3E0910201F091030109958091C0004C
:1039B00087FFE9CF8091C600992787FD90951F91D9
:1039C0000F91FF90EF900895982F8091C00085FF90
:1039D000FCCF9093C60008950E94B81C803271F00D
:1039E000809104018F5F80930401853009F0089570
:1039F000E0910201F09103010995089584E10E948C
:103A0000E41C80E10E94E41C08951F93182F0E947B
:103A1000B81C803269F0809104018F5F80930401AB
:103A2000853079F4E0910201F0910301099509C014
:103A300084E10E94E41C812F0E94E41C80E10E942A
:103A4000E41C1F910895282F882351F090E0809165
:103A5000C00087FFFCCF8091C6009F5F2917B9F790
:103A60000895CFEFD4E0DEBFCDBF94B714BE8091F0
:103A700060008861809360001092600091FFEFC148
:103A800089E18093C4001092C50088E18093C10051
:103A900086E08093C2005098589A259A81E00E944F
:103AA000511C0E94B81C8033B9F18133C1F18034BC
:103AB00009F455C0813409F45BC0823409F46AC04A
:103AC000853409F46DC0803539F1813509F404C1BC
:103AD000823511F1853509F4BDC0863509F4B3C0CE
:103AE000843609F463C0843709F4FCC0853709F4CF
:103AF000CEC0863709F44AC0809104018F5F80935D
:103B00000401853071F6E0910201F09103010995FD
:103B10000E94B81C803349F60E94EC1CC2CF0E9460
:103B2000B81C803249F784E10E94E41C81E40E94C1
:103B3000E41C86E50E94E41C82E50E94E41C80E20D
:103B40000E94E41C89E40E94E41C83E50E94E41CBA
:103B500080E50E94E41C80E10E94E41CA2CF0E9448
:103B6000B81C8638C8F20E94B81C0E94EC1C99CF81
:103B70000E94B81C803809F4ABC0813809F4A4C095
:103B8000823809F49DC0883909F496C080E00E940B
:103B9000051D87CF84E10E94231D0E94EC1C81CF6C
:103BA00085E00E94231D0E94EC1C7BCF0E94B81C64
:103BB000809309020E94B81C8093080280910C0235
:103BC0008E7F80930C020E94B81C853429F480916A
:103BD0000C02816080930C0280910802909109028E
:103BE000892B09F042C00E94B81C803209F084CFB2
:103BF00080910C0280FFC5C080910802909109025B
:103C00000097D1F02091060130910701E8E0F1E042
:103C1000AC014E0F5F1FF999FECF32BD21BD8191DE
:103C200080BDFA9AF99A2F5F3F4FE417F50799F78D
:103C3000309307012093060184E10E94E41C80E197
:103C40000E94E41C2ECF84E00E94231D80E00E948D
:103C5000051D27CF0E94B81C809306010E94B81C46
:103C6000809307010E94EC1C1CCFC0E0D0E008E06C
:103C700011E00E94B81CF80181938F012196809178
:103C8000080290910902C817D90798F3ACCF0E9497
:103C9000B81C803209F030CF84E10E94E41C8EE130
:103CA0000E94E41C84E90E94E41C86E00E94E41C5B
:103CB00080E10E94E41CF5CE83E00E94051DF1CE58
:103CC00080E10E94051DEDCE81E00E94051DE9CE38
:103CD00082E00E94051DE5CE0E94EC1C88E08093E6
:103CE0006000FFCF0E94B81C809309020E94B81C9C
:103CF000809308020E94B81C853409F4BEC08091EC
:103D00000C028E7F80930C02809106019091070136
:103D1000880F991F90930701809306010E94B81C99
:103D2000803209F0BECE84E10E94E41C809108023A
:103D300090910902009709F4BBCFC0E0D0E0E09178
:103D40000601F091070120910C0220FF8EC0F99925
:103D5000FECFF2BDE1BDF89A80B50E94E41CE0916F
:103D60000601F09107013196F0930701E0930601F7
:103D700080910802909109022196C817D90718F37B
:103D800097CF8091070187FD66C010920B0280914A
:103D9000060190910701880F991F90930701809366
:103DA00006018091080280FF09C08091080290916D
:103DB000090201969093090280930802F894F999F8
:103DC000FECF1127E0910601F0910701C8E0D1E094
:103DD0008091080290910902103091F400915700EF
:103DE00001700130D9F303E000935700E89500918A
:103DF000570001700130D9F301E100935700E895B5
:103E0000099019900091570001700130D9F301E039
:103E100000935700E8951395103498F011270091FE
:103E2000570001700130D9F305E000935700E89581
:103E30000091570001700130D9F301E10093570060
:103E4000E8953296029709F0C7CF103011F002962C
:103E5000E5CF1124F1CE81E080930B0298CFE09161
:103E60000201F091030109950BCE21FF0CC03196A0
:103E7000F0930701E09306017FCF80910C028160EF
:103E800080930C024BCF84910E94E41C8091080225
:103E900090910902E0910601F0910701E8CF0F939C
:103EA0001F930E94B81C182F0E94E41C0E94B81C8B
:103EB000082F0E94E41C11362CF0175501363CF0F7
:103EC000075508C01033D4F310530136CCF7003334
:103ED0000CF000531295107F100F812F992787FD4A
:103EE00090951F910F9108951F93282F992787FD73
:103EF0009095807F907095958795959587959595E8
:103F00008795959587958A304CF0982F995A822FEE
:103F10008F708A304CF0182F195A08C0982F905D76
:103F2000822F8F708A30BCF7182F105D892F0E9466
:0C3F3000E41C812F0E94E41C1F910895E6
:023F3C00800003
:0400000300003800C1
:00000001FF
